:0300000002001EDD
:03001B000200627E
:10001E0075812153E88075985043878043D880C2FC
:10002E00ACD299C298758D38758B387588007589E4
:10003E002275A90975B90075A800D2ABD2AFD28EC0
:10004E0012007EF5F843F880700500000080F10084
:10005E00000080EC1200C512006932C0D0A20592D9
:10006E00E8A20492E9A20692EEA20892EAD0D02269
:10007E00120098D2051201B33002F8C2054008D220
:10008E00041200E4C2042202017F750932751500C4
:10009E00C204C205C206C207C208D200D203D201F0
:1000AE00C202221201CB30020B1201CB200205E557
:1000BE0015700122740822200105D50A02D201D53D
:1000CE000913750932200005D50802D20020030558
:1000DE00D50B02D20322780C7A007B001201B320DA
:1000EE000205500602017C02017FEB0B9002079382
:1000FE0012018F30020302017F120117700AE5F020
:10010E00F608E515B43AE3E422A915B9070302018E
:10011E0078B90E03020178B9140630E55102017860
:10012E00B91C0820D010547F020178B9230B20D0BF
:10013E0005543F020178020182B929061201850297
:10014E000178B92C06120185020178B93106120127
:10015E0085020178B9391A1201851201B3200211F4
:10016E00C5F0EA3330D005020182F5F0E4227401C5
:10017E0022740422740222A2D0C0E0EA33FAD0E044
:10018E0022F5F0C0F0E41201B3300203D0F02213D6
:10019E00D5F0F3D0F0C0E07408C395F0F5F0D0E0E0
:1001AE0003D5F0FC22C0E01201CB20020D75080F22
:1001BE00C2003000FD1201F99206D0E022750B64E8
:1001CE00C2031201F920032040F8750B64C203121A
:1001DE0001F920031350F8C20805153002077515F2
:1001EE0000D208C202D20722D20222A2EF40087524
:1001FE000A05C2013001FDB32207070608070603F0
:02020E000508E1
:00000001FF
